:1000000050C0B0C269C068C067C066C065C064C087
:1000100063C062C061C060C05FC05EC05DC00501FA
:100020000906A101050719E029E715002501750159
:1000300095088102950175082565190029658100DB
:10004000C00403090412036F0062006400650076B7
:10005000002E0061007400160345006100730079F2
:10006000004C006F0067006700650072001201100D
:100070000100000008424231E100010102000109D3
:1000800002220001010080190904000001030000A0
:100090000009210101000122230007058103080056
:1000A0000A0011241FBECFE5D1E0DEBFCDBF10E0B6
:1000B000A0E6B0E0EAE1FAE002C005900D92A836B1
:1000C000B107D9F710E0A8E6B0E001C01D92A73A49
:1000D000B107E1F739D0A0C493CF80916D00882398
:1000E00011F499E301C090E08F5F80936D0010924E
:1000F0006A0090936B000895FC018AE690E090936B
:100100008C0080938B00808180768032D1F4818155
:10011000813021F4E2DF82E090E00895823049F4FA
:100120008CE690E090938C0080938B0081E090E0CF
:1001300008958A3031F4838180936C0080E090E0F0
:10014000089580E090E00895CF93DF93A0E0B0E0C1
:10015000C2D3802D8F3F09F081BFB89A20E083EB96
:1001600091EF0197F1F72F5F2431C9F7B898BC9A46
:10017000C19A88E190E02EE00FB6F894A89581BD71
:100180000FBE21BD8BE080BF86E792E090936F00A9
:1001900080936E0079D07894CAE6D0E0A895A0D07C
:1001A0008091620084FF08C080916D00823020F44D
:1001B00094DF62E0CE0172D008B602FEEFCF84E099
:1001C00088BF8091680090916900019690936900C2
:1001D0008093680020916E0030916F008217930722
:1001E000E8F26AD38D5E944F90936F0080936E0017
:1001F000109269001092680010926D00CFCFDF92CC
:10020000EF92FF920F931F93CF93DF9380E8D82E46
:10021000FF24C0E0D0E0EF2CED0CE1BE90D18C01CA
:1002200089E0043318070CF4FE2CD6942196C830CC
:10023000D10589F7FA94F1BEF394CF2DD0E0219641
:1002400010C07DD18453994097FF03C0909581954C
:100250009F4F8017910714F4F1B68C0181B78F5F1F
:1002600081BF81B790E0C817D9075CF7F1BE81B7AD
:10027000A0E0B0E0082E37D3DF91CF911F910F910E
:10028000FF90EF90DF90089585B7836085BF8BB7AF
:1002900080648BBF83EC80937D0008951F93DC0105
:1002A000162F8091620084FF07C080917D0098E83E
:1002B000892780937D0003C08AE580936200912F97
:1002C000EEE7F0E002C08D9181939150E0F7612F4D
:1002D0008EE790E030D11C5F109362001F9108956B
:1002E0000F931F93CF93DF9390918D0019160CF00D
:1002F000A8C020918A00809189008D3209F099C0B0
:100300008AE5809361009B3009F093C0CDE9D0E08D
:10031000C21BD1098881807609F07CC02BE730E0D0
:1003200010927B008981882341F410927C003093E5
:100330008C0020938B0092E070C0853021F48A817C
:1003400080938E0065C0863009F046C08B81813075
:1003500019F48DE690E01BC0823041F48FE790E005
:1003600090938C0080938B0092E25AC0833001F509
:100370008A81882341F481E490E090938C008093FB
:100380008B0094E04DC0813041F485E490E090937F
:100390008C0080938B0092E143C0823009F03FC013
:1003A00087E590E090938C0080938B0096E138C0B5
:1003B000813241F481E990E090938C0080938B002E
:1003C00099E02EC0823259F58EE190E090938C0036
:1003D00080938B0093E224C0883039F480E990E068
:1003E00090938C0080938B000CC0893021F48A811B
:1003F000809390000DC08A3031F430938C002093AC
:100400008B0091E00AC08B3019F483EC80937D005F
:1004100090E003C0CE0170DE982F20E802C090E08B
:1004200020EC8F81882339F48E81891720F4982F4E
:1004300002C090E020E82093710090936000109239
:100440008D008091610084FF45C0809160008F3FE6
:1004500009F440C0182F893008F018E0811B809300
:1004600060008091710080FF02C003EC01C00BE4CA
:100470008F5F8093710020918B0030918C0086FDFE
:1004800005C0912FF901A3E7B0E00DC0912FF9014C
:10049000A3E7B0E003C084918D9331969150D8F7D3
:1004A00004C081918D939150E0F7C901810F911D96
:1004B00090938C0080938B00612F83E790E03BD07A
:1004C000183019F08FEF80936000009372001C5F6A
:1004D000109361009AE086B3857031F49150D9F79A
:1004E00010928E001092880010E0992309F411E018
:1004F00080917000811729F0112309F480DE109398
:100500007000DF91CF911F910F910895A82FB92FFF
:1005100080E090E041E050EA60956F5F58F42D91E3
:1005200038EF82279795879510F0842795273F5FAE
:10053000C8F3F3CF0895EADF8D939D930895A6E065
:1005400088279927AA9569F00197E1F3B099FCCF24
:10055000B09BFECF81E09927A6B3019611F0A5705C
:10056000D9F70895CF93CFB7CF93B09BFECFB09B71
:100570000BC0B09B09C0B09B07C0B09B05C0B09B2F
:1005800003C0B09B01C0D5C00F92DF93C0918A0019
:10059000DD27CF56DF4F012EB09B03C0DF910F90B8
:1005A000E6CF2F930F931F934F932FEF4F6F06B309
:1005B00000FB20F95F933F9350E03BE065C016B32A
:1005C0000126502950FDC89556B3012700FB25F997
:1005D0002F7306B3B1F05027102710FB26F906B28F
:1005E0002230F0F000C016B3012700FB27F90126E6
:1005F000502906B22430E8F54F77206816B3000082
:10060000F6CF50274F7D206206B2102F000000C0A9
:1006100006B300265029102710FB26F906B2E2CFB8
:100620004F7B06B3206400C0DACF01265029157035
:1006300006B269F14E7F2160012F16B328C0002653
:1006400050294D7F06B22260102F29C00126502963
:100650004B7F06B22460012F2DC016B3012650290E
:10066000477F2860000006B22EC04F7E06B320618F
:1006700030C0422706B3499300265029102706B2FE
:100680004FEF10FB20F9297F16B379F2157059F15D
:100690000126502906B2012700FB21F9237F06B36A
:1006A00071F2002650293150D0F006B2102710FB0D
:1006B00022F9277E16B351F201265029012700FBAB
:1006C00006B223F92F7C49F2000006B3102710FB75
:1006D00024F90026502906B22F7939F270CF10E4A0
:1006E0001ABF002719C03B503195C31BD04010E4FE
:1006F0001ABF0881033C09F10B34F9F020918800FE
:100700001981110F1213EDCF4A81441F093651F19F
:100710000D3211F0013E29F700938F003F915F9158
:100720004F911F910F912F91DF910F90CAB7C6FD86
:100730001CCFCF91CFBFCF91189500918F00002390
:1007400069F310918D00112379F534307AF13093EB
:100750008D000093890010918A003BE0311B30939B
:100760008A0024C000918D000130F4F40AE54F7036
:1007700049F43091610034FD1AC000936100C2E772
:10078000D0E019C03091620034FD11C000936200C6
:10079000CDE7D0E010C0052710E000C021C005273C
:1007A00010E0C89508BB14C03AE501C032ED032E35
:1007B000C0E0D0E032E017B31560C09A08B317BBB1
:1007C00055E020E84FEF20FF052708BB2795179538
:1007D0001C3F28F700004552B0F720FF052727955A
:1007E00008BB17951C3FB8F629913A9561F70A7F27
:1007F00010918E00110F08BBC250D04011F0109321
:10080000880010E41ABF016017B31A7F402F4A7F97
:1008100054E05A95F1F708BB17BB48BB7FCFA0E067
:10082000B0E0E4E1F4E0A7C0EC01688179818A815D
:100830009B81611571058105910549F484E2A82E1B
:1008400089EDB82E8BE5C82E87E0D82E02C05B015B
:100850006C01C601B5012DE133EF41E050E068D0F5
:1008600027EA31E440E050E04AD07B018C01C60128
:10087000B5012DE133EF41E050E05AD0CA01B90192
:1008800024E13BE040E050E03AD0E61AF70A080BDA
:10089000190BD801C70117FF04C081509040A04038
:1008A000B04888839983AA83BB839F77EAE0CDB75A
:1008B000DEB77DC0B4DF089583E690E0B0DF089531
:1008C000A0E0B0E08093630090936400A093650083
:1008D000B09366000895E199FECFBFBBAEBBE09A2E
:1008E00011960DB20895E199FECFBFBBAEBB0DBA14
:1008F00011960FB6F894E29AE19A0FBE0895FF2779
:10090000EE27BB27AA2760FF04C0A20FB31FE41F76
:10091000F51F220F331F441F551F96958795779516
:10092000679589F70097760771F7CF01BD010895A4
:1009300097FB092E05260ED057FD04D04BD00AD0C8
:10094000001C38F450954095309521953F4F4F4FFE
:100950005F4F0895F6F790958095709561957F4F5C
:100960008F4F9F4F08952F923F924F925F926F92B9
:100970007F928F929F92AF92BF92CF92DF92EF922F
:10098000FF920F931F93CF93DF93CDB7DEB7CA1BB0
:10099000DB0B0FB6F894DEBF0FBECDBF09942A88DB
:1009A000398848885F846E847D848C849B84AA8483
:1009B000B984C884DF80EE80FD800C811B81AA8110
:1009C000B981CE0FD11D0FB6F894DEBF0FBECDBFDB
:1009D000ED010895A1E21A2EAA1BBB1BFD010DC05B
:1009E000AA1FBB1FEE1FFF1FA217B307E407F507DF
:1009F00020F0A21BB30BE40BF50B661F771F881FBB
:100A0000991F1A9469F760957095809590959B0150
:0A0A1000AC01BD01CF010895FFCF36
:080A1A00FF5A5A010000000020
:00000001FF
